:020000040000FA
:10000000000080308A00712820000B1D1528AA0AE4
:10001000AA0F0C287116F20A2B082A0222000318D4
:100020000C11031C0C150B1170282700931C3D2884
:1000300020000130F700FE30970083309600111049
:1000400018146400111832288C1C212803100C1875
:100050000314F70D031834286400111832288C1883
:100060002C282128701537287708AD00F0141810B7
:100070002700931020000B10702820008C1A4728AE
:10008000BE30200096019700111018146C2818102B
:1000900011186628AE1A4D286C28DE3017022E1B68
:1000A0005328B10C5428B20C031C6C282E1B5A2860
:1000B0002E176C280310310CAF000310B20CB20CD9
:1000C000320CB000AE122E13AE176C284030B100C7
:1000D0001030B200AE162E132700931220000B1022
:1000E000090021009618762896141614031E482C31
:1000F0006400F0302100990020002030840080014D
:10010000840A841F7F2823008C018E010E158E1413
:100110008E150C160E1422008C018E0121000C117C
:100120000E1224008C018E018C140C148C166400A9
:100130000830210095000130210097002000950132
:100140000B118B1627009214200064008C1EA5282A
:1001500027009216270091162700930120000B100C
:100160008B158B17210019309D0020309E00220036
:100170008C309700220088309800153099002200BA
:1001800094309100133092009430930081309400A9
:1001900064001518C828200012132000FF309B00AF
:1001A00025000C3093009101043020009C002000B9
:1001B00091106400911CDA289110250095131516F2
:1001C00021008E1220000230AB0001302224AC004E
:1001D0002C090319AC012C08023C031CF128023045
:1001E000AC00FF30A00000302224F900F919F0150E
:1001F00002302224A50003302224A7003B24210042
:100200009D142500951B702C7A211E23A10A211C08
:1002100012292508260203191229031C1129A603F5
:100220001229A60AEE21A000F43EA400F522AB009C
:10023000200091106400911C1B299110A60803193D
:100240002329121F3429121322000E162000A2089F
:10025000031D2D29A30803194429A303A31F44291F
:100260000330A300A203442922000E12200022081A
:100270002402031C4129A30A231D4429A301A20A25
:1002800044292408A200A30122082500910020008F
:10029000230E30390C3825009300200091106400A3
:1002A000911C5029200820009B002000AE1BC92370
:1002B000F01C5E292D08A500F015F010711E012913
:1002C0006223701C01290C1C01298C1C01298B1133
:1002D00022000C148C1021000C108C10200025081A
:1002E000042421000C148C14270093010B108B158F
:1002F0007010012921000E1A8C29F30803199A297C
:10030000721F9A290E16F40A73087402031C9A29A4
:1003100070170530F4009A29701B9129721F0E1274
:100320009A29741C9829721BF40B9A2970139A2924
:10033000721FF40320000800250803190800F03E8E
:10034000031C013003190130A500F015BC21080081
:100350002509031908002508103E0318FF30A500E1
:10036000F015BC210800FF30A500F015BC210800E5
:10037000A501F015BC210800023022242502031932
:10038000C5292508230093002A24003022242300B5
:100390009319CC2993152A24033022242702031908
:1003A000D5292708230093002A2408007308013C5C
:1003B000031CF303B723080004307302031CF30A81
:1003C000B723080081308A007308E93E03188A0ABF
:1003D00082000234143426344034663481308A007A
:1003E0002608F53E03188A0A8200FF34FF34FE34E3
:1003F000FD34FC34FB34FB34FA34F934F834F7348C
:10040000F634F634F534F434F334F234F134F134B0
:10041000F034EF34EE34ED34EC34EC34EB34EA34D5
:10042000E934E834E834E734E634E534E434E334FA
:10043000E334E234E134E034DF34DE34DE34DD341E
:10044000DC34DB34DA34D934D934D834D734D63444
:10045000D534D534D434D334D234D134D034D03468
:10046000CF34CE34CD34CC34CB34CB34CA34C9348D
:10047000C834C734C634C634C534C434C334C234B3
:10048000C134C134C034BF34BE34BD34BD34BC34D7
:10049000BB34BA34B934B834B834B734B634B534FC
:1004A000B434B334B334B234B134B034AF34AE3422
:1004B000AE34AD34AC34AB34AA34AA34A934A83445
:1004C000A734A634A534A534A434A334A234A1346B
:1004D000A034A0349F349E349D349C349B349B3490
:1004E0009A349934983497349634963495349434B5
:1004F000933492349234913490348F348E348D34DA
:100500008D348C348B348A348934883488348734FD
:100510008634853484348334833482348134803423
:100520007F347F347E347D347C347B347A347A3447
:10053000793478347734763475347534743473346C
:1005400072347134703470346F346E346D346C3492
:100550006C346B346A3469346834673467346634B5
:1005600065346434633462346234613460345F34DB
:100570005E345D345D345C345B345A345934583401
:100580005834573456345534543454345334523424
:10059000513450344F344F344E344D344C344B344A
:1005A0004A344A344934483447344634453445346F
:1005B0004434433442344134413440343F343E3493
:1005C0003D343C343C343B343A34393438343734B9
:1005D00037343634353434343334323432343134DD
:1005E00030342F342E342D342D342608FB002C08C3
:1005F000FF3EFA01FB0C0318FA07FA0CFB0C031878
:10060000FA07FA0CFB0C0318FA07FA0CFB0C031898
:10061000FA07FA0CFB0C0318FA07FA0CFB0C031888
:10062000FA07FA0CFB0C0318FA07FA0CFB0C031878
:10063000FA07FA0CFB0C7A08023E0800701E242B05
:1006400021009D147012602B21009D18602BF01A60
:10065000552BF01D3C2B21001C0820002702031CF9
:10066000003C083C03184E2BF011003022242300DC
:10067000931D4E2B93112A242808A70021001C0843
:100680002000A800A707A70CA7080319A70A270896
:10069000250203194E2B2708A5007014F0160D3003
:1006A00021009D0020007016602B21001C082000F6
:1006B000A907A90C2908F012193021009D00701615
:1006C0002000080020008C186C2BF11A742BF50FF9
:1006D000742BF114F116742BF11A722B0A30750277
:1006E00003187114F112F5010C187D2B711B852B69
:1006F000F60F852BF1157117852B711B832B0A3093
:100700007602031871157113F6017112F01BA22BFA
:10071000F11C8D2B711B972BB82171189C21F11D99
:10072000942BF11A972BB3217119A821AF2B27080D
:10073000013C031DAF2BF0170130F300B723A501D7
:10074000F011AF2BF11CA72B711BB42BAB2BF11DA0
:10075000AB2BF11AB42B7118D6217119DC21711051
:100760007111F110F1110800F013F301AF2B0430F7
:100770007302031CBD2B0430F300E221AC000130F6
:1007800022242C020319C82B2C08230093002A24AE
:100790000800AE130A302F020318D12B2F0AF900DC
:1007A000E12B10302F02031DD72BA821E12B113094
:1007B0002F02031DDD2B9C21E12B14302F02031986
:1007C000B8210800F9016400E52BE62BE72BE82BA4
:1007D000E92BEA2BEB2BEC2BED2BEE2BEF2BF02B5D
:1007E000F12BF22BF32BF42BF52BF62BF72BF82B0D
:1007F000F92BFA2BFB2BFC2BFD2BFE2BF90FE32BFC
:10080000FF3E0318E32B0800F8008030F90078055C
:10081000031D1A24031912240310F90C7908031C70
:10082000072C080022008C100C10162C172C8C148E
:100830002000080022008C100C141E2C1F2C8C147D
:1008400020000800230091001513951315141308B8
:100850002000080023001513951315158B13553030
:100860009600AA30960095148B1715116400951800
:10087000362C2000080022000E165030E2230E1203
:100880005030E2230E165030E2230E1220000800F2
:100890008B133A30210099002100FF308C008E002C
:1008A0000E1222000E120830E2230E160130E2234F
:1008B000482C8B133A30210099002100FF308C0026
:1008C0008E000E1222000E120830E2230E160130A6
:1008D000E2230E120130E2230E160130E223592CDE
:1008E0008B133A30210099002100FF308C008E00DC
:1008F0000E1222000E120830E2230E160130E223FF
:100900000E120130E2230E160130E2230E120130E6
:10091000E2230E160130E223702C00340034FF3F36
:10092000FF3FFF3FFF3FFF3FFF3FFF3FFF3FFF3FD7
:10093000FF3FFF3FFF3FFF3FFF3FFF3FFF3FFF3FC7
:10094000FF3FFF3FFF3FFF3FFF3FFF3FFF3FFF3FB7
:10095000FF3FFF3FFF3FFF3FFF3FFF3FFF3FFF3FA7
:020000040001F9
:04000E00DCFFFF3BD9
:00000001FF
